S123F8003838380102060C1080204E6F20524453207369676E616C20524453206465636F4F
S123F82064657220666F7220206D696E692D7465726D696E616C2020534D204E6F2050542B
S123F840592020204E657773202041666661697273202020496E666F20202053706F7274EE
S123F86020204564756361746520204472616D61202043756C7475726520536369656E63CB
S123F8806520205661726965642020506F70204D202020526F636B204D202045617379203A
S123F8A04D204C69676874204D20436C6173736963734F74686572204D2057656174686530
S123F8C0722046696E616E6365204368696C6472656E20536F6369616C2052656C6967699E
S123F8E06F6E50686F6E6520496E2054726176656C204C6569737572652020204A617A7AD0
S123F9002020436F756E747279204E6174696F6E204D204F6C646965732020466F6C6B204D
S123F9204D20446F63756D656E74202054455354202020416C61726D20218E00FF8600B73F
S123F940100186FFB71007BDFBC1CEF818860F971486009724BDFBD3CEF828861F97148618
S123F960009724BDFBD3CE00C8BDFBAB0926FA8601BDFC9B7F00137F00157F00167F0025E1
S123F9807F0026863ACE0029A702B6100A84024D26129625810A27037C00258105260DBDFC
S123F9A0FCE520E696254D27037A0025BDFD25961181D826D59612810326CF7600007600A4
S123F9C0017600027600037600007600017600027600039601970896029709BDFD16BDFD5B
S123F9E025961181D426A396128103269D76000076000176000276000376000076000176E9
S123FA0000027600039601970A9602970BBDFD16BDFD259611815C270781CC27037EF98A1C
S123FA20961281032707810227037EF98A7600007600017600027600037600007600017679
S123FA4000027600039601970C9602970DBDFD16BDFD259611815827037EF98A961281022C
S123FA6027037EF98A7600007600017600027600037600007600017600027600039601976D
S123FA800E9602970FDE089C15275A8601BDFC9B4F97267F0013DF15CE0008BDFC59CE00DB
S123FAA01786049714860C9724BDFBD3960A8403D60BC4E00404C3F83A8F86179714860018
S123FAC09724BDFBD3CE000A1F00F0037EFAE5CEF838960B84084D27010886019714860A2B
S123FAE09724BDFBD3CE000A1F00F0037EFB46D613810F275118CE0013D60BC403C100269A
S123FB0004181C0001C1012604181C0002C1022604181C0004C1032604181C0008584FC3CD
S123FB20001B8FD60EE700D60F08E7009613810F27037EFB46CE001B8608971486019724F2
S123FB40BDFBD37EFB46CE000AA60084F8814027037EFBA8CE000DA600CE000EE600840189
S123FB60C4F004545454D727CE000FA600841F441F002009D6279727D0271720029B2797D9
S123FB8027CE000EA600CE000FE600840FC4C00505972818CE0027BDFC32CE0029861597F4
S123FBA014860A9724BDFBD37EF98A183C18CE06DA180926FC18383918CE1800180926FC2F
S123FBC039CEF800A600BDFC9BBDFBB8088CF80926F23936373C183C18CE001418E600C419
S123FBE00FCB01D723181E0010228680BDFC9B9624270A8614BDFC9B7A002426F2A6007ABB
S123FC0000232728BDFCBA0820F3202086C0BDFC9B962427E88614BDFC9B7A002426F2A6F3
S123FC20007A00232706BDFCBA0820F318383833323918A600164FCE000A028FCB30D729BB
S123FC408FCB30D72A18A601164FCE000A028FCB30D72C8FCB30D72D39A60084F0444444DD
S123FC6044810A25028B078B309717A600840F810A25028B078B309718A60184F00C4444F9
S123FC804444810A25028B078B309719A601840F810A25028B078B30971A39B710048600B5
S123FCA0B710038608B710038600B71003BDFCD0393CCE00210926FD3839B710048604B738
S123FCC01003860CB710038604B71003BDFCB1393CCE0025BDFCB10926FA38393CCE00017C
S123FCE00926FD3839363796268101271A8601BDFC9B7F0015CEF809860F971486019724B7
S123FD00BDFBD386019726333239CE100A1E0001F91F0001FC39368619BDFD0ABDFD2F4A51
S123FD204D26F63239BDFD0ABDFD2FBDFD4A390C368608B4100A4D260220010D79000379CB
S123FD400002790001790000323936373C7F00117F0012D603D707D602D706D601D705D680
S123FD6000D7049605D604C403CE00001F070104881BC8031F070204888FC8031F070404C5
S123FD8088A7C8021F07080288F71F07100488EEC8011F07200488DCC8031F0740048801D2
S123FDA0C8021F07800488BBC8011F0601048876C8031F0602048855C8031F060404881331
S123FDC0C8031F060804889FC8031F0610048887C8021F06200288B71F064004886EC80171
S114FDE01F06800488DCC802D7129711383332393B95
S123FFD6FDF0FDF0FDF0FDF0FDF0FDF0FDF0FDF0FDF0FDF0FDF0FDF0FDF0FDF0FDF0FDF037
S10DFFF6FDF0F93AF93AF93AF93A44
S9030000FC
